:020000040800F2
:100000006009002045010008F9100008611000088F
:10001000F5100008B1010008432F0008000000009F
:10002000000000000000000000000000052600089D
:10003000F10D000800000000A5210008512800086B
:100040005F0100085F0100085F0100085F01000810
:100050005F0100085F0100085F0100085F01000800
:100060005F0100085F0100085F0100085F010008F0
:100070005F0100085F0100085F0100085F010008E0
:100080005F0100085F0100085F0100085F010008D0
:100090005F0100085F0100085F0100085F010008C0
:1000A0005F0100085F0100085F0100085F010008B0
:1000B0005F010008B92800085F0100085F0100081F
:1000C0005F0100085F0100085F0100085F01000890
:1000D0005F010008992A0008F52A0008D92B0008BA
:1000E0005F0100085F0100085F0100085F01000870
:1000F0005F0100085F0100085F0100085F01000860
:100100005F0100085F0100085F0100085F0100084F
:100110005F0100085F0100085F0100085F0100083F
:100120005F0100085F0100085F0100085F0100082F
:10013000DFF80CD000F02AF80048004749300008EA
:10014000600900200648804706480047FEE7FEE7B2
:10015000FEE7FEE7FEE7FEE7FEE7FEE7FEE7FEE777
:100160005528000831010008D2B201E000F8012B47
:10017000491EFBD270470022F6E710B513460A4627
:1001800004461946FFF7F0FF204610BD064C074D08
:1001900006E0E06840F0010394E807009847103457
:1001A000AC42F6D3FFF7C8FFAC330008CC330008ED
:1001B00000BFFEE710B502460B460020002104E018
:1001C000545C0444E0B24C1CE1B29942F8DBC443F5
:1001D000E0B2441CE0B210BDFEB5002000900190DA
:1001E000029000F057FF3A4800780A2822D1394897
:1001F000007839490978884218D13648407836491C
:100200004978884212D13348007A3349097A8842C2
:100210000CD13048407A3049497A884206D12F487B
:10022000008840F400402D49088003E0142129484B
:10023000FFF7A1FF2948008800F40040002846D0BD
:10024000274800210160017126480160017126489C
:100250000160017125480160017100202149087089
:100260001C48007948701B4840798870194880798B
:10027000C8701848C079087100201D4908701948D5
:10028000407848701748807888701648C078C870E1
:1002900014480079087113484078040611488078A2
:1002A00005041048C0780602601930440D490979E8
:1002B000471801200F49087000F0ECFE00200449A7
:1002C00008700649088014210248FFF754FFFEBD5C
:1002D00009000020D40100200C0000200A000020AA
:1002E00034000020160000203C00002041000020C7
:1002F0001B0000204900002010B588B07F4800781E
:10030000012838D100207D490870FC207C49087004
:10031000112048707B48007888707A484078C8700F
:100320007848807808717748C078487175480079B6
:10033000887107217248FFF73DFF7149C87100209D
:1003400071490860FF22E121012001F079FE0823B4
:100350006B4AA821012001F035FE012001F0B8F917
:1003600001206A49C1F8A40169490870002069495F
:10037000088000F08FFE6748008840F6B831884258
:100380007BDC00F087FE604884380068002857D185
:1003900000F080FE6946012001F0F2FD044620468F
:1003A00002F07EF95CA002F085F904F040004028DC
:1003B000EDD100208DF80A000721684600F019FDF4
:1003C00055A002F077F99DF801004E49097888425E
:1003D00054D19DF802004B49497888424ED19DF88E
:1003E000030048498978884248D19DF8040045496E
:1003F000C978884242D19DF805004249097988426E
:100400003CD14348007801281BD141480078401C6A
:100410003F49087012203A49487007213848FFF7D1
:10042000C9FE3749C8710020374908600823344A9B
:10043000A821012001F0C6FD01203449C1F8A40122
:1004400058E00020324908700E21344800F0D1FCF9
:1004500031A002F02FF932480178012001F092F921
:1004600010202E4948700E212C4802F00DF92DA0C5
:1004700002F020F9012008B010BD16E0002022494A
:10048000086011201E49487007211D48FFF792FEA1
:100490001B49C87108230A46A821012001F092FDDA
:1004A00001201A49C1F8A40124E000201549087070
:1004B00048708870C87008711B490870487088704F
:1004C000C87008711949087048708870C870087140
:1004D0001749087048708870C870087130200F493B
:1004E00048700E210D4802F0CFF812A002F0E2F899
:1004F0000120C0E700F0CEFD0020BCE74600002050
:100500004A00002034000020A481214200802142C2
:100510008A000020260000200A000000C8030020F6
:10052000320000204F4B0A00410000201B00002039
:1005300016000020333030300A00000010B588B0BB
:100540004B480088B0F5FA6F71DA4A480068002815
:100550006ED100F09FFD6946012001F011FD0446B7
:1005600004F04000402875D100208DF80A009DF865
:10057000010078B99DF8020060B99DF8030048B900
:1005800000203D49087048708870C87008710120CB
:1005900008B010BD39480078072803D037480078E4
:1005A0000D280FD10020344908709DF800004870D4
:1005B0009DF8010088709DF80200C8709DF8030046
:1005C000087145E02D480078082810D19DF80100F9
:1005D000294908709DF8020048709DF80300887052
:1005E0009DF80400C8709DF80500087130E02348AC
:1005F0000078092803D0214800780E2819D100205E
:100600001D4908709DF8010080F0530048709DF866
:10061000020080F0430088709DF8030080F04400E1
:10062000C8709DF8040080F05800087110E014E0D4
:1006300010E00020104908709DF8010048709DF8F6
:10064000020088709DF80300C8709DF804000871CE
:1006500001209DE700F01EFD08E00020064908701B
:1006600048708870C8700871012091E700208FE7FA
:100670003A00002020812142410000203200002069
:1006800010B500F007FDFE480078082829D1FD4884
:100690000078752825D1FB484078702821D1F94889
:1006A000807864281DD1F748C078612819D1F548B1
:1006B0000079742815D1F3484079652811D10020BC
:1006C000EF49087000BFF048006800F4E060EF49AF
:1006D0000843001DEC490860BFF34F8F00BF00BF07
:1006E000FEE7E8480078752807D0E6480078FA2841
:1006F00003D00020E249087010BDE14800780E28C0
:1007000000DAF9E7DE480078401EDE49085CFB2885
:1007100000D0F1E7DB48807AA02804D1D8480078DF
:10072000152800D0E8E7D64800780E281ED1D54815
:100730000078FA2814D1D348407BFB2810D1D44844
:10074000008840F40040D24908800020CC4908705D
:100750000E21CC4800F04DFBCEA001F0ABFF4AE0EB
:100760000020C7490870CA49088044E0C44800789E
:1007700015281ED1C3480078FA2814D1C148007D3D
:10078000FB2810D1C248008840F40040C0490880CE
:100790000020BB4908701521BA4800F02AFBBDA013
:1007A00001F088FF27E00020B5490870B8490880AB
:1007B00021E0B348007811281DD1B2480078FA280A
:1007C00014D1B048007CFB2810D1B148008840F417
:1007D0000040AF4908800020A94908701121A948AC
:1007E00000F007FBABA001F065FF04E00020A44986
:1007F0000870A7490880A648008800F40040002837
:1008000071D000F047FC9F488079A34988719D48CA
:10081000C179A148C1719B48017A9F4801729948EA
:10082000417A9D4841729748807A9B498872084670
:1008300080799A4988719848C1799848C1719648D9
:10084000017A964801729448417A944841729248DC
:10085000807A94284CD018DC732834D00CDC2528FE
:1008600025D004DC21281AD022287DD11BE026289F
:1008700021D07128F9D122E0742828D075282AD0F7
:1008800078282CD08228F0D12EE0A03809286BD20D
:10089000DFE800F0329CA0F5F4F3F2F1F000002064
:1008A0007D498872DFE100207B498872DBE100200E
:1008B00079498872D7E1002077498872D3E1002016
:1008C00075498872CFE1002073498872CBE100201E
:1008D00071498872C7E100206F498872C3E1002026
:1008E0006D498872BFE1C2E100206B498872BAE1AC
:1008F000002069498872B6E10020614908706648A5
:100900008079674988716448C1796548C1716248D6
:10091000017A634801726048417A614841725E48D9
:10092000807A5F4988725748407B5B4948735548D5
:10093000817B594881735348C17B5748C1735148E3
:10094000017C554801744F48417C534841744D48DF
:10095000407B544908704B48807B48704948C07BB5
:1009600088704848007C00E07CE1C8704548407CC5
:10097000087101204C49087000204C490880012072
:1009800000F0A6FE4AA001F095FE04E0FFF7B4FCDB
:10099000044604B100E0F9E700BF45A001F08AFE7B
:1009A00000204549087048708870C8700871434934
:1009B000087048708870C8700871414908704870A4
:1009C0008870C8700871344988724CE1002032493F
:1009D000887248E13B48007830B93848002101600E
:1009E00001710120374908703448407848B93348CC
:1009F000807830B93148C07818B93048007900B9EA
:100A000031E100201E490870234880792E49887101
:100A10002148C1792C48C1711F48017A2A480172C6
:100A20001D48417A284841721B48807A26498872BD
:100A30000120C87206200873002048731F480178FF
:100A4000214881731D4841781F48C1731B48817834
:100A50001D4801741948C1781B4841741748017931
:100A600019488174162101F00FFE322002F098FA25
:100A700016212BE0ADE0F1E0ECE0E7E03AE038E011
:100A8000030000200C0100200CED00E00000FA053E
:100A9000040000200A000000000300209C02002047
:100AA000C80300203400002046000020260000205B
:100AB000303030300A000000410000201B000020D0
:100AC000160000202B00002064030020694800F07D
:100AD00090F9AFF2400001F0EDFD0020664908708A
:100AE00048708870C87008716449087064498872D9
:100AF000B9E0B8E00020634908706348017801203C
:100B000000F040FE00206149088061A001F0D2FDA4
:100B100004E0FFF713FD044604B100E0F9E700BF6D
:100B20005BA001F0C7FD564880795249887154484E
:100B3000C1795048C1715248017A4E4801725048FB
:100B4000417A4C4841724E48807A4A498872012065
:100B5000C87206200873002048734F480178454842
:100B600081734D4841784348C1734B48817841486F
:100B700001744948C1783F484174474801793D486C
:100B80008174162101F080FD322002F009FA16214D
:100B9000384800F02EF93FA001F08CFD00203E49BE
:100BA000087048708870C8700871334908704870C0
:100BB0008870C87008713949087048708870C870AA
:100BC00008712D4800210160017100202C498872B4
:100BD00049E03348407B2C490870294880793149E5
:100BE00088712748C1792F48C1712548017A2D485D
:100BF00001722348417A2B4841722148807A294961
:100C00008872012048700E21264801F03DFD3220F7
:100C100002F0C6F91C4800782349088001F0FCFC6A
:100C200000201D49087048708870C870087112490A
:100C3000087048708870C87008711849087048704A
:100C40008870C87008710E4988720CE000200C4949
:100C5000887208E000200A49887204E000200849F0
:100C6000887200E000BF00BF00201049088000BF6C
:100C700042E50000640300201B0000202B00002040
:100C80000003002003000020320000203A00002072
:100C9000343434340A0000004100002016000020E3
:100CA0000C0100202C04002034050020040000204A
:100CB000FA204A49087010204870002088700021EE
:100CC0004648C1700171417100204449887100217A
:100CD0004248C1710172417200204049C87400212C
:100CE0003E480175FB203D494875FA203C49087093
:100CF000102048700020887000213948C1700171AF
:100D0000417100203649887100213548C171017256
:100D100041720020324981F84B000021304880F8B0
:100D20004C10FB202E4981F84D00FA202D49087007
:100D3000102048700020887000212A48C17001717D
:100D4000417100202749887100212648C171017234
:100D5000417200202349C872002122480173FB2000
:100D600020494873FA20204908701020487000205C
:100D7000887000211C48C1700171417100201A491E
:100D8000887100211848C171017241720020164912
:100D9000C874002114480175FB2013494875FA20D6
:100DA00012490870102048700020887000210F48F8
:100DB000C1700171417100200C49887100210B48FC
:100DC000C1710172417200200849C87200210748B0
:100DD0000173FB2005494873704700009C02002006
:100DE000000300202C04002064030020C80300201E
:100DF00070472DE9F04104460E460DE02578281194
:100E000000F030F9074601F04BFC284600F02AF9C3
:100E1000074601F045FC641C301EA6F10101CEB26C
:100E2000ECD1BDE8F081000030B5044604254FF454
:100E3000302000F06FF80546042D17D10C480069EA
:100E400040F002000A49086108464461006940F028
:100E5000400008614FF4302000F05CF8054604487B
:100E6000006941F6FD71084001490861284630BD1E
:100E70000020024004200B49C96801F0010109B1BA
:100E800001200EE00749C96801F0040109B1022000
:100E900007E00449C96801F0100109B1032000E02E
:100EA00004207047002002400348006940F08000A1
:100EB00001490861704700000020024070B50446F7
:100EC0000D460426F00200F025F80646042E11D146
:100ED0000948006940F00100074908612580F002D7
:100EE00000F018F806460448006941F6FE71084013
:100EF00001490861304670BD0020024002480349A4
:100F0000486003484860704723016745002002405D
:100F1000AB89EFCD00B502460423FFF7ABFF0346D4
:100F200003E0FFF7A7FF0346521E012B01D1002A61
:100F3000F7D102B90523184600BD2DE9F04102465C
:100F400000250026002000230024002791F803C07C
:100F50000CF00F0591F803C00CF0100CBCF1000F61
:100F600003D091F802C04CEA050591F800C0BCF12D
:100F7000000F31D0146800202BE04FF0010C0CFA68
:100F800000F3B1F800C00CEA03069E4220D18300B2
:100F90004FF00F0C0CFA03F7BC4305FA03FC4CEAC4
:100FA000040491F803C0BCF1280F06D14FF0010CE6
:100FB0000CFA00FCC2F814C00AE091F803C0BCF1BE
:100FC000480F05D14FF0010C0CFA00FCC2F810C01C
:100FD000401C0828D1D31460B1F800C0BCF1FF0F49
:100FE00034DD546800202EE000F1080C4FF00108B9
:100FF00008FA0CF3B1F800C00CEA03069E4221D1B6
:1010000083004FF00F0C0CFA03F7BC4305FA03FC06
:101010004CEA040491F803C0BCF1280F05D100F19B
:10102000080C08FA0CF8C2F8148091F803C0BCF15F
:10103000480F07D100F1080C4FF0010808FA0CF82E
:10104000C2F81080401C0828CED35460BDE8F0815F
:10105000416170470161704701460A8890B270474C
:1010600000BFFEE70146002001F00F02092A04DC60
:1010700001F00F0202F1300003E001F00F023732FD
:10108000D0B270474CF6CC40014908607047000070
:101090000030004010B500F013F810BD70B50546E3
:1010A0000C4645F2555000F01FF8284600F010F8A5
:1010B000204600F013F800F003F8FFF7E3FF70BDDF
:1010C0004AF6AA200149086070470000003000403D
:1010D00001494860704700000030004001498860C5
:1010E0007047000000300040014908607047000070
:1010F0000030004000BFFEE7704700007CB50546A9
:1011000012A103C9CDE900010821284601F052FAD5
:1011100005236A463021284600F054FF05236A461D
:101120001021284600F0BEFE002406E01DF8040051
:10113000A52800D003E0601CC4B2052CF6DB00BF7C
:10114000052C01D001207CBD0020FCE7A5A5A5A5AC
:10115000A500000008B501211C2001F035F8402051
:10116000ADF8000010208DF8030003208DF8020078
:1011700069463248FFF7E1FE40213048FFF76AFF39
:101180001020ADF8000069462D48FFF7D6FE10216B
:101190002B48FFF75FFF8020ADF8000048208DF856
:1011A000030003208DF8020069462448FFF7C5FEBE
:1011B0004FF40070ADF8000010208DF803000320FC
:1011C0008DF8020069461D48FFF7B7FE4FF4007125
:1011D0001A48FFF73FFF4FF48050ADF80000694612
:1011E0001648FFF7AAFE4FF480511448FFF732FF6C
:1011F0004FF48070ADF8000048208DF80300032004
:101200008DF8020069460D48FFF797FE01F000F9DE
:1012100001F0BCF800200B49086001200A49C1F820
:101220009001002007490C31086001200749C1F8EE
:10123000B0010821002001F0BDF908BD000C0140FB
:101240000008014098812142000021420080214293
:1012500010B5044602222321204600F0F1FE0523AA
:101260001E4A2A21204600F0ADFE05231B4A3021EC
:10127000204600F0A7FE3F222121204600F0E0FE9C
:1012800001222221204600F0DBFE1A2225212046E1
:1012900000F0D6FE24222621204600F0D1FE0F22A7
:1012A0002021204600F0CCFE0A223121204600F009
:1012B000C7FE01223D21204600F0C2FE00223C2153
:1012C000204600F0BDFE70222721204600F0B8FE27
:1012D000FF22E221204600F0B3FE10BD613300087A
:1012E00010B5044602222321204600F0A9FE042363
:1012F0001E4A2A21204600F065FE04231B4A3021A5
:10130000204600F05FFE30222121204600F098FEAA
:1013100001222221204600F093FE122225212046A0
:1013200000F08EFE24222621204600F089FE0F22A6
:101330002021204600F084FE08223121204600F0C2
:101340007FFE01223D21204600F07AFE00223C2152
:10135000204600F075FE70222721204600F070FE26
:10136000FF22E221204600F06BFE10BD98330008FA
:1013700010B5044602222321204600F061FE04231A
:101380001E4A2A21204600F01DFE04231B4A30215C
:10139000204600F017FE30222121204600F050FEAA
:1013A00001222221204600F04BFE28222521204642
:1013B00000F046FE0C222621204600F041FE0F22BE
:1013C0002021204600F03CFE06223121204600F07C
:1013D00037FE01223D21204600F032FE00223C2152
:1013E000204600F02DFE70222721204600F028FE26
:1013F000FF22E221204600F023FE10BD8E330008BC
:1014000010B5044602222321204600F019FE0423D1
:101410001E4A2A21204600F0D5FD04231B4A302114
:10142000204600F0CFFD30222121204600F008FEAA
:1014300001222221204600F003FE1622252120460B
:1014400000F0FEFD04222621204600F0F9FD0F22C7
:101450002021204600F0F4FD08223121204600F032
:10146000EFFD01223D21204600F0EAFD00223C2153
:10147000204600F0E5FD70222721204600F0E0FD27
:10148000FF22E221204600F0DBFD10BDA73300085B
:1014900010B5044602222321204600F0D1FD04238A
:1014A0001E4A2A21204600F08DFD04231B4A3021CC
:1014B000204600F087FD30222121204600F0C0FDAB
:1014C00001222221204600F0BBFD332225212046A7
:1014D00000F0B6FD04222621204600F0B1FD0F22C7
:1014E0002021204600F0ACFD09223121204600F0E9
:1014F000A7FD01223D21204600F0A2FD00223C2153
:10150000204600F09DFD70222721204600F098FD26
:10151000FF22E221204600F093FD10BD8433000835
:1015200010B5044602222321204600F089FD052340
:101530001E4A2A21204600F045FD05231B4A302182
:10154000204600F03FFD3F222121204600F078FD9B
:1015500001222221204600F073FD1222252120467F
:1015600000F06EFD04222621204600F069FD0F22C6
:101570002021204600F064FD0A223121204600F09F
:101580005FFD01223D21204600F05AFD00223C2152
:10159000204600F055FD70222721204600F050FD26
:1015A000FF22E221204600F04BFD10BD523300081F
:1015B00010B5044602222321204600F041FD0523F8
:1015C0001E4A2A21204600F0FDFC05231B4A30213B
:1015D000204600F0F7FC30222121204600F030FDAB
:1015E00001222221204600F02BFD12222521204637
:1015F00000F026FD21222621204600F021FD0F22A9
:101600002021204600F01CFD0A223121204600F056
:1016100017FD00223D21204600F012FD01223C2151
:10162000204600F00DFD70222721204600F008FD25
:10163000FF22E221204600F003FD10BD43330008E5
:1016400010B5044601222321204600F0F9FC0523B1
:101650001E4A2A21204600F0B5FC05231B4A3021F2
:10166000204600F0AFFC30222121204600F0E8FCAB
:1016700001222221204600F0E3FC192225212046E8
:1016800000F0DEFC04222621204600F0D9FC0F22C7
:101690002021204600F0D4FC06223121204600F013
:1016A000CFFC01223D21204600F0CAFC00223C2153
:1016B000204600F0C5FC70222721204600F0C0FC27
:1016C000FF22E221204600F0BBFC10BD7033000871
:1016D00010B504461CB900202749086003E000202B
:1016E00025490C31086001222321204600F0A8FC86
:1016F0000323224A2A21204600F064FC0323204AC7
:101700003021204600F05EFC01222121204600F01D
:1017100097FC01222221204600F092FC2A2225215A
:10172000204600F08DFC04222621204600F088FC93
:101730000F222021204600F083FC06223D21204676
:1017400000F07EFC01223C21204600F079FC702252
:101750002721204600F074FCFF22E221204600F001
:101760006FFC1CB901200449086003E00120024914
:101770000C31086010BD0000988121423933000807
:101780003433000870B504460D461CB900203849B2
:10179000086003E0002036490C310860142D5BD24C
:1017A000DFE805F00A0E12161A1E22262A2E3236FD
:1017B0003A3E42464A4E52562046FFF7F9FE4BE06B
:1017C000204600F097FA47E0204600F023FB43E074
:1017D0002046FFF7A5FE3FE0204600F0FBF93BE086
:1017E000204600F0D7F837E02046FFF731FD33E020
:1017F000204600F0A7F92FE0204600F0C3FA2BE0C6
:101800002046FFF71DFF27E0204600F033F823E0D5
:10181000204600F027FA1FE0204600F073F81BE096
:101820002046FFF735FE17E02046FFF709FF13E0DB
:101830002046FFF79DFD0FE0204600F03BF90BE04E
:101840002046FFF74DFD07E0204600F0EBF803E0EF
:101850002046FFF7D5FD00BF00BF1CB90120044999
:10186000086003E0012002490C31086070BD0000EF
:101870009881214210B5044602222321204600F01F
:10188000DFFB04231E4A2A21204600F09BFB042391
:101890001B4A3021204600F095FB302221212046B2
:1018A00000F0CEFB01222221204600F0C9FB2022BD
:1018B0002521204600F0C4FB20222621204600F0EE
:1018C000BFFB0F222021204600F0BAFB0822312165
:1018D000204600F0B5FB01223D21204600F0B0FB80
:1018E00000223C21204600F0ABFB7022272120463D
:1018F00000F0A6FBFF22E221204600F0A1FB10BD74
:101900007533000810B5044602222321204600F05A
:1019100097FB04231E4A2A21204600F053FB042390
:101920001B4A3021204600F04DFB30222121204669
:1019300000F086FB01222221204600F081FB1222CA
:101940002521204600F07CFB24222621204600F0A1
:1019500077FB0F222021204600F072FB0A22312162
:10196000204600F06DFB01223D21204600F068FB7F
:1019700000223C21204600F063FB702227212046F4
:1019800000F05EFBFF22E221204600F059FB10BD73
:101990007F33000810B5044602222321204600F0C0
:1019A0004FFB05231E4A2A21204600F00BFB05238E
:1019B0001B4A3021204600F005FB30222121204621
:1019C00000F03EFB01222221204600F039FB1222CA
:1019D0002521204600F034FB24222621204600F059
:1019E0002FFB0F222021204600F02AFB0A22312162
:1019F000204600F025FB01223D21204600F020FB7F
:101A000000223C21204600F01BFB702227212046AB
:101A100000F016FBFF22E221204600F011FB10BD72
:101A20005C33000810B5044602222321204600F052
:101A300007FB04231E4A2A21204600F0C3FA042390
:101A40001B4A3021204600F0BDFA302221212046D9
:101A500000F0F6FA01222221204600F0F1FA1422C9
:101A60002521204600F0ECFA04222621204600F031
:101A7000E7FA0F222021204600F0E2FA0A22312163
:101A8000204600F0DDFA01223D21204600F0D8FA80
:101A900000223C21204600F0D3FA70222721204664
:101AA00000F0CEFAFF22E221204600F0C9FA10BD74
:101AB0009D33000810B5044602222321204600F081
:101AC000BFFA04231E4A2A21204600F07BFA042391
:101AD0001B4A3021204600F075FA30222121204691
:101AE00000F0AEFA01222221204600F0A9FA1222CB
:101AF0002521204600F0A4FA24222621204600F0C9
:101B00009FFA0F222021204600F09AFA0822312164
:101B1000204600F095FA01223D21204600F090FA7F
:101B200000223C21204600F08BFA7022272120461B
:101B300000F086FAFF22E221204600F081FA10BD73
:101B40009333000810B5044601222321204600F0FB
:101B500077FA05231E4A2A21204600F033FA05238E
:101B60001B4A3021204600F02DFA30222121204648
:101B700000F066FA01222221204600F061FA1022CC
:101B80002521204600F05CFA04222621204600F0A0
:101B900057FA0F222021204600F052FA0622312166
:101BA000204600F04DFA01223D21204600F048FA7F
:101BB00000223C21204600F043FA702227212046D3
:101BC00000F03EFAFF22E221204600F039FA10BD73
:101BD0006633000810B5044602222321204600F097
:101BE0002FFA05231E4A2A21204600F0EBF905238F
:101BF0001B4A3021204600F0E5F930222121204601
:101C000000F01EFA01222221204600F019FA1222C9
:101C10002521204600F014FA24222621204600F037
:101C20000FFA0F222021204600F00AFA0822312163
:101C3000204600F005FA01223D21204600F000FA7E
:101C400000223C21204600F0FBF97022272120468B
:101C500000F0F6F9FF22E221204600F0F1F910BD74
:101C60005733000810B5044602222321204600F015
:101C7000E7F904231E4A2A21204600F0A3F9042391
:101C80001B4A3021204600F09DF9302221212046B8
:101C900000F0D6F901222221204600F0D1F91C22C1
:101CA0002521204600F0CCF924222621204600F0F0
:101CB000C7F90F222021204600F0C2F90822312165
:101CC000204600F0BDF901223D21204600F0B8F980
:101CD00000223C21204600F0B3F970222721204643
:101CE00000F0AEF9FF22E221204600F0A9F910BD74
:101CF0007A33000810B5044603222321204600F061
:101D00009FF905231E4A2A21204600F05BF905238E
:101D10001B4A3021204600F055F93F222121204660
:101D200000F08EF93F222221204600F089F9282276
:101D30002521204600F084F904222621204600F0C7
:101D40007FF90B222021204600F07AF90A22312166
:101D5000204600F075F901223D21204600F070F97F
:101D600000223C21204600F06BF9702227212046FA
:101D700000F066F9FF22E221204600F061F910BD73
:101D80004833000810B5044601222321204600F004
:101D900057F903231E4A2A21204600F013F9032392
:101DA0001B4A3021204600F00DF930222121204627
:101DB00000F046F901222221204600F041F92A22B2
:101DC0002521204600F03CF904222621204600F07F
:101DD00037F90F222021204600F032F90722312165
:101DE000204600F02DF900223D21204600F028F980
:101DF00001223C21204600F023F9702227212046B1
:101E000000F01EF9FF22E221204600F019F910BD72
:101E10006B33000810B5044603222321204600F04E
:101E20000FF905231E4A2A21204600F0CBF805238E
:101E30001B4A3021204600F0C5F8302221212046DF
:101E400000F0FEF801222221204600F0F9F81022CD
:101E50002521204600F0F4F804222621204600F037
:101E6000EFF80F222021204600F0EAF80A22312163
:101E7000204600F0E5F801223D21204600F0E0F880
:101E800000223C21204600F0DBF87022272120466A
:101E900000F0D6F8FF22E221204600F0D1F810BD74
:101EA0004D3300082DE9F0478046894615461E4609
:101EB000B8F1000F16D10020174908604946404686
:101EC00000F024FB0746002406E0FF21404600F016
:101ED0001DFB2855601CC4B2B442F6DB01200E493C
:101EE000086015E000200D4908604946404600F0B2
:101EF0000DFB0746002406E0FF21404600F006FBEC
:101F00002855601CC4B2B442F6DB012003490860C6
:101F10003846BDE8F087000090012142B08121429F
:101F200070B505460E4685B9002011490860314656
:101F3000284600F0EBFAFF21284600F0E7FA0446B5
:101F400001200C49C1F890010FE000200A49086007
:101F50003146284600F0DAFAFF21284600F0D6FA8A
:101F6000044601200549C1F8B001204670BD0000BB
:101F70009001214200002142B08121420080214293
:101F800070B506460D461021304600F013FB0721C0
:101F90003046FFF7C5FF044622462721304600F0B1
:101FA0004FF804F0400050B10A232A466121304620
:101FB000FFF778FFFF22E221304600F041F820468B
:101FC00070BD00002DE9F0478046894615461E4643
:101FD000B8F1000F16D10020174908604946404665
:101FE00000F094FA0746002406E015F8011B40466D
:101FF00000F08CFA601CC4B2B442F6DB01200E493A
:10200000086015E000200D4908604946404600F090
:102010007DFA0746002406E015F8011B404600F053
:1020200075FA601CC4B2B442F6DB012003490860B3
:102030003846BDE8F087000090012142B08121427E
:102040002DE9F04104460E46154684B90020114999
:1020500008603146204600F059FA074629462046D6
:1020600000F054FA01200C49C1F890010FE0002063
:102070000A4908603146204600F048FA07462946DA
:10208000204600F043FA01200549C1F8B001384666
:10209000BDE8F0819001214200002142B08121423F
:1020A0000080214208B54FF4C06000F071F826208E
:1020B0008DF8000001208DF8010002208DF802004B
:1020C00001208DF80300684600F02AF827208DF8DB
:1020D000000001208DF801008DF802008DF803004A
:1020E000684600F01DF825208DF8000000208DF8CE
:1020F000010001208DF802008DF80300684600F011
:102100000FF81D208DF8000000208DF801008DF8DB
:10211000020001208DF80300684600F001F808BDB8
:1021200070B5002100230F22C47804B3154C246835
:1021300004F4E064C4F5E064210AC1F10403CA4078
:10214000447804FA03F184781440214309010E4CC9
:102150000678A155047804F01F050124AC400578E9
:102160006D11AD0005F1E025C5F8004109E00478E6
:1021700004F01F050124AC40044D0678761145F8A3
:10218000264070BD0CED00E000E400E080E100E0DE
:1021900002490143024A1160704700000000FA053D
:1021A0000CED00E07047000029B1064AD2690243F5
:1021B000044BDA6104E0034AD2698243014BDA61DD
:1021C000704700000010024029B1064A926902439C
:1021D000044B9A6104E0034A92698243014B9A617D
:1021E000704700000010024070B5012144F20D005C
:1021F000FFF7EAFF01210220FFF7D6FF042000F0DD
:1022000013FB1249B1F1807F00D31DE021F07F4024
:10221000401E4FF0E022506150170F22002807DACD
:1022200013071D0E0A4B00F00F04241F1D5503E079
:1022300013071C0E074B1C5400BF00204FF0E02278
:1022400090610720106100BF70BD000080A90300ED
:1022500018ED00E000E400E070B500210023002448
:10226000002200252C4E766806F00C0121B10429CD
:1022700005D0082921D105E0284E066020E0274E30
:1022800006601DE0244E766806F47013224E7668D0
:1022900006F48034022606EB93431CB9204E5E43BD
:1022A000066009E01C4E7668C6F34046751C1B4E5E
:1022B000B6FBF5F65E43066002E0184E066000BF0E
:1022C00000BF154E766806F0F0010909154E725CE4
:1022D0000668D6404660104E766806F4E061090A4A
:1022E000104E725C4668D64086600B4E766806F4E7
:1022F0006051C90A0B4E725C4668D640C660064EF5
:10230000766806F44041890B074E725CC668B6FBDE
:10231000F2F6066170BD00000010024000127A0063
:1023200000093D0090000020A000002010B586B0FC
:102330000024142101A8FDF71EFF0A2201A9084864
:1023400000F012F800BF07E001A810F81400054AD9
:1023500002F81400601CC4B20A2CF5DB06B010BDF4
:10236000000003084805002070B504460D461646D7
:10237000002300BF07E02046FEF76EFE25F813009D
:10238000A41C581CC3B2B342F5DB70BD00B587B0C6
:10239000012141F20500FFF717FFE020ADF818001A
:1023A00018208DF81B0003208DF81A0006A9164886
:1023B000FEF7C3FDE0211448FEF74CFE0020ADF807
:1023C00004004FF48270ADF806000020ADF808005C
:1023D000ADF80A00ADF80C004FF40070ADF80E0037
:1023E0001820ADF810000020ADF812000720ADF85D
:1023F000140001A9054800F06BF80121034800F022
:102400004DF807B000BD0000000801400030014059
:1024100000B587B001218803FFF7C6FE012109201E
:10242000FFF7D2FE4FF46040ADF8180018208DF889
:102430001B0003208DF81A0006A91648FEF77DFD43
:102440004FF460411348FEF705FE0020ADF804008C
:102450004FF48270ADF806000020ADF80800ADF82A
:102460000A00ADF80C004FF40070ADF80E00182013
:10247000ADF810000020ADF812000720ADF81400F0
:1024800001A9054800F024F80121034800F006F8EE
:1024900007B000BD000C01400038004021B10288A7
:1024A00042F04002028004E002884FF6BF731A40F7
:1024B000028070470246002013890B400BB10120B7
:1024C00000E000207047014688897047818170478D
:1024D00010B50022028802F441520B884C88234335
:1024E0008C882343CC8823430C8923434C89234382
:1024F0008C892343CC8923431A430280838B4FF278
:10250000FF74234083830B8A038210BD2DE9F041C1
:1025100006460F4626BB06E0601CC4B2C82C02DB90
:102520000020BDE8F08102212048FFF7C3FF00280A
:10253000F2D039461D48FFF7C9FF002405E0601CB2
:10254000C4B2C82C01DB0020EBE701211748FFF7DC
:10255000B1FF0028F3D01548FFF7B5FFC5B222E060
:1025600005E0601CC4B2C82C01DB0020D9E70221C1
:102570000F48FFF79FFF0028F3D039460C48FFF7BC
:10258000A5FF002405E0601CC4B2C82C01DB0020BC
:10259000C7E701210648FFF78DFF0028F3D0044864
:1025A000FFF791FFC5B22846BBE7000000300140AD
:1025B0000038004070B505460C467DB90F480088CC
:1025C0004FF6C77108400D4908800846008820432F
:1025D000088001210A48FFF761FF0EE008480088E3
:1025E0004FF6C77108400649088008460088204316
:1025F000088001210248FFF751FF70BD0030014003
:1026000000380040704770B504460D462946204604
:10261000FEF754FC70BD000010B586B000241421F4
:1026200001A8FDF7A8FD00BF07E00B4830F8140033
:1026300001A921F81400601CC4B20A2CF5DB07487C
:1026400000F0EAF80A2201A9044800F009F800F0B5
:102650007AFC06B010BD000034050020000003081D
:102660002DE9F04105460F461646002400BF07E05D
:1026700037F814102846FFF7C6FFAD1C601CC4B223
:10268000B442F5DBBDE8F08170B504460D46034A5F
:102690002946204600F028F870BD000000380140AF
:1026A00010B504460249204600F00EF810BD0000A7
:1026B0000044004010B504460249204600F02DF8C1
:1026C00010BD00000044004070B504460D4600BF38
:1026D0008021284600F064FB0028F9D021462846D6
:1026E00000F02BFC012070BD2DE9F04104460D46A1
:1026F000164614B90120BDE8F0810AE014F8017B08
:1027000031463846FFF7E0FF08B90020F3E7681EBE
:1027100085B2002DF2D10120EDE770B504460E46DA
:102720000CB9012070BD11E014F8015B0A2D06D12F
:1027300031460D20FFF7C8FF08B90020F2E7314607
:102740002846FFF7C1FF08B90020EBE720780028F2
:10275000EAD10120E6E710B500F002F810BD000054
:102760000CB50020019000902A48006840F48030A9
:102770002849086000BF2748006800F40030009036
:102780000198401C0190009818B90198B0F5A06F0D
:10279000F1D12048006800F4003010B10120009011
:1027A00001E0002000900098012831D119484068CC
:1027B00018494860084640684860084640684860D4
:1027C0000846406820F47C1048600846406840F4A1
:1027D000981048600846006840F08070086000BFAC
:1027E0000C48006800F000700028F9D009484068E3
:1027F00020F00300074948600846406840F00200A6
:10280000486000BF0348406800F00C000828F9D178
:102810000CBD00000010024010B50446FEF76EFB30
:102820002046FEF701FB10BD042808D14FF0E0213F
:10283000096941F004014FF0E022116107E04FF017
:10284000E021096921F004014FF0E0221161704795
:102850007047000010B51448006840F001001249AC
:10286000086008464068114908400F49486008461A
:1028700000680F4908400C4908600846006820F4C9
:10288000802008600846406820F4FE0048604FF44D
:102890001F0088600020C862FFF75DFF4FF00060F6
:1028A0000449086010BD0000001002400000FFF85D
:1028B000FFFFF6FE08ED00E010B50121204800F012
:1028C0007EF800283AD001211D4800F069F81D4823
:1028D0000088401C1B4908801B480088401C1A497E
:1028E00008801A480088401C184908801848007859
:1028F000C0B14FF400711748FEF7ACFB16480088D2
:10290000401C1549088008460088B0F5C87F09DBDF
:102910004FF400710F48FEF79BFB00200E49088022
:102920000B4908700948008841F28831884202D179
:1029300000200649088001200849087010BD0000E9
:1029400000040040260000203A000020280000205B
:102950002C000020001001402E0000202A00002042
:102960003EB505460C4601210220FFF71DFCADF8DF
:102970000450ADF800400020ADF80600ADF80200AC
:102980006946064800F036F801221146034800F077
:1029900027F80121014800F006F83EBD0004004080
:1029A000CA430282704721B1028842F001020280CC
:1029B00004E002884FF6FE731A400280704730B57B
:1029C0000246002000230024158A05EA01039589A8
:1029D00005EA010413B10CB1012000E0002030BD74
:1029E0001AB183890B43838102E083898B438381FE
:1029F00070470000002202881D4B98420ED01D4BEC
:102A000098420BD0B0F1804F08D01B4B984205D0B4
:102A10001A4B984202D01A4B984204D14FF68F734A
:102A20001A404B881A43174B984207D0164B9842CE
:102A300004D04FF6FF431A40CB881A4302808B889C
:102A400083850B8803850A4B98420BD0094B98422B
:102A500008D00E4B984205D00D4B984202D00D4B3A
:102A6000984201D10B7A03860123838270470000CC
:102A7000002C0140003401400004004000080040E8
:102A8000000C0040001000400014004000400140D5
:102A9000004401400048014010B540F22551124861
:102AA00000F08BF988B140F225510F4800F0CFF8C3
:102AB0000D4800F03DFAC4B20C480D490978445461
:102AC0000B480078401C0A4908700821064800F0AD
:102AD00067F9012806D10821034800F0AFF8024841
:102AE00000F026FA10BD0000003801400C01002063
:102AF0000300002010B540F22551124800F05DF9A6
:102B000088B140F225510F4800F0A1F80D4800F0BF
:102B10000FFAC4B20C480D49097844540B480078A8
:102B2000401C0A4908700821064800F039F90128BC
:102B300006D10821034800F081F8024800F0F8F9B6
:102B400010BD000000440040F40400208D0000206F
:102B500010B586B0044601210520FFF735FB0121A1
:102B60004804FFF721FB0420ADF8140003208DF882
:102B7000160018208DF8170005A91548FEF7DDF995
:102B80000820ADF8140004208DF8170005A910489E
:102B9000FEF7D3F901940020ADF80800ADF80A0063
:102BA000ADF80C00ADF810000C20ADF80E0001A936
:102BB000084800F051F9012240F22551054800F083
:102BC00026F90121034800F051F806B010BD0000BD
:102BD000000801400044004010B540F2255114485F
:102BE00000F0EBF8B0B140F22551114800F02FF899
:102BF0000F4800F09DF9C4B20E480F4909784454BB
:102C00000D480078401C0C4908700846007800F018
:102C10000F0008700821064800F0C2F8012806D10C
:102C20000821034800F00AF8014800F081F910BDBE
:102C300000480040D40100200900002001F4007287
:102C4000B2F5007F00D100BFCA430280704710B5C3
:102C50000022002340F66A14A14200D100BF0A12EC
:102C600001249440A3B2DC43048010BD21B18289C9
:102C700042F40052828104E082894DF6FF731A40CB
:102C80008281704700B585B0012144F20400FFF74E
:102C90009BFA4FF40070ADF8000003208DF802009D
:102CA00018208DF8030069463948FEF746F94FF4BD
:102CB0008060ADF8000004208DF8030069463448B8
:102CC000FEF73BF94FF4164001900020ADF80800E4
:102CD000ADF80A00ADF80C00ADF810000C20ADF80E
:102CE0000E0001A92B4800F0B7F8012240F225514F
:102CF000284800F08CF801212648FFF7B7FF012192
:102D00008804FFF751FA01210820FFF75DFA4FF41C
:102D10008060ADF8000003208DF8020018208DF8C7
:102D2000030069461C48FEF708F94FF40060ADF84F
:102D3000000004208DF8030069461748FEF7FDF8EF
:102D40004FF4965001900020ADF80800ADF80A004D
:102D5000ADF80C00ADF810000C20ADF80E0001A984
:102D60000E4800F079F801A90C4800F075F801222E
:102D700040F22551094800F04AF801210748FFF7C1
:102D800075FF40210348FFF759FF05B000BD000063
:102D90000008014000380140000C0140004800409C
:102DA00002460020B1F5007F00D100BF13880B4020
:102DB0000BB1012000E00020704770B502460024EE
:102DC00000230025002040F66A16B14200D100BF62
:102DD000C1F3421501F01F03012606FA03F3012D8A
:102DE00002D19689334006E0022D02D1168A334083
:102DF00001E0968A33400C12012606FA04F4168884
:102E0000344013B10CB1012000E0002070BDF0B5DA
:102E10000346002400260025002040F66A17B94228
:102E200000D100BF1846C1F3421401F01F0601276C
:102E300007FA06F5012C01D10C3004E0022C01D177
:102E4000103000E014301AB107682F43076002E029
:102E50000768AF430760F0BD2DE9F04786B005462F
:102E60000E460024A24600BFA1460027B08900B14B
:102E700000BF2F462C8A4CF6FF700440F0880443B4
:102E80002C82AC894EF6F3100440B0883189084397
:102E9000718908430443AC81AC8A4FF6FF4004407B
:102EA000B0890443AC8201A8FFF7D6F91F488742D6
:102EB00002D1DDF810A001E0DDF80CA0A88900F433
:102EC000004040B10AEBCA0000EB0A10316849002B
:102ED000B0FBF1F807E00AEBCA0000EB0A1031681A
:102EE0008900B0FBF1F86420B8FBF0F00401200980
:102EF000642101FB1089A88900F4004040B1322010
:102F000000EBC900B0FBF1F000F00700044308E05B
:102F1000322000EB09106421B0FBF1F000F00F004B
:102F200004432C8106B0BDE8F08700000038014062
:102F300001468888C0F308007047C1F30802828008
:102F4000704700BFFEE710B5FDF7AEFF10BD0000F3
:102F5000014A024900F013B8CD2F0008A400002058
:102F600002E008C8121F08C1002AFAD17047704752
:102F7000002001E001C1121F002AFBD170472DE99A
:102F8000F04116460F460446002503E03946B04797
:102F9000641C6D1C20780028F8D12846BDE8F0811B
:102FA00010B502460BE0C82007E0122101E04B1EDD
:102FB00099B20029FBDC431E98B20028F5DC131EF1
:102FC000A2F10104A2B2EED110BD000070B504461A
:102FD0000D46E0B20549088000BF40210348001FAC
:102FE000FFF7DEFE0028F8D0204670BD043801400F
:102FF00008B501211020FFF7E7F80120ADF8000027
:1030000010208DF8030003208DF8020069460D485A
:10301000FDF793FF01210B48FEF71CF84FF40070F9
:10302000ADF8000010208DF8030003208DF8020099
:1030300069460448FDF781FF4FF400710148FEF72F
:1030400007F808BD00100140FFF7CEF8FFF72AF897
:1030500040F271210420FEF721F8FEF71BF841F63B
:103060001F410920FFF77CFCFFF7C2FFFFF70AFEB4
:103070004FF4E130FFF76CFDFEF76CF8FEF70AF84D
:1030800002E04FA0FFF764FF0120FEF737F80028A9
:10309000F7D1FDF70DFEFDF7FDFF4D480068C04379
:1030A0004C49C1F88001C820FFF77AFF4948D0F8A1
:1030B0008001C0434749C1F88001062146A0FDF7C1
:1030C00098FE47A0FFF7F6FAFDF7E4FF45A0FFF7EB
:1030D0003FFF0120FEF7FCFAFFF728F94A48007885
:1030E0004A4908700846007814285BD2DFE800F0EF
:1030F0000A0E12161A1E22262A2E32363A3E424650
:103100004A4E525642A0FFF723FF4BE043A0FFF781
:103110001FFF47E044A0FFF71BFF43E045A0FFF778
:1031200017FF3FE046A0FFF713FF3BE047A0FFF784
:103130000FFF37E049A0FFF70BFF33E04AA0FFF78E
:1031400007FF2FE04CA0FFF703FF2BE04DA0FFF798
:10315000FFFE27E04EA0FFF7FBFE23E04FA0FFF7A6
:10316000F7FE1FE051A0FFF7F3FE1BE054A0FFF7AE
:10317000EFFE17E056A0FFF7EBFE13E058A0FFF7B5
:10318000E7FE0FE05AA0FFF7E3FE0BE05CA0FFF7BD
:10319000DFFE07E05EA0FFF7DBFE03E060A0FFF7C5
:1031A000D7FE00BF00BF0120614908703220FFF741
:1031B000F7FE03E0FDF710F8FDF762FAFAE700000A
:1031C00054686520322E3447204572726F72210098
:1031D0008001224200002242313233343536000071
:1031E0000A0000000A5043B6D4C2EBC8EDBCFECDC5
:1031F000A8D3C3B0E6B1BE56322E332D32303139AA
:10320000303630350A00000048050020320000202A
:10321000BDADCEF7D0ADD2E90D0A0000CCECB2A81E
:10322000D0ADD2E90D0A0000D4C6C4CFD0ADD2E9EA
:103230000D0A0000B9F3D6DDD0ADD2E90D0A0000C9
:10324000CBC4B4A8D0ADD2E90D0A0000C4DAC3C91A
:10325000B9C5D0ADD2E90D0A00000000B0B2BBD5AF
:10326000D0ADD2E90D0A0000C9BDCEF7F6CEC5B586
:10327000D0ADD2E90D0A000056434F4DB2E2CAD498
:103280000D0A0000C1C9C4FEB5E7D0C50D0A000093
:10329000C1C9C4FED2C6B6AF0D0A00005470D7A88B
:1032A000D3C3D0ADD2E90D0A00000000C4DAC3C90F
:1032B000B9C5D2C6B6AFD0ADD2E90D0A0000000044
:1032C000B9E3CEF7D2C6B6AFD0ADD2E90D0A000051
:1032D000CBC4B4A8B5E7D0C5D0ADD2E90D0A000083
:1032E000B8A3BDA8D5E6D7C6D0ADD2E90D0A000077
:1032F000CBD5D6DDC4BEC0BCD0ADD2E90D0A00002E
:10330000D6D8C7ECD2C6B6AFD0ADD2E90D0A000010
:10331000C9BDCEF7D2C6B6AFD0ADD2E90D0A000016
:10332000B8CACBE0D2C6B6AFD0ADD2E90D0A000024
:103330002B000020344310100134431010013320BF
:103340000D547933200D54793443101001011010BD
:1033500043343223ABBA013412BBAA01341286754E
:10336000014656431000346E4610013443101001DC
:10337000862C95010136E4A7BC014218BAE8013455
:103380001286750133200D5400862C9500005A4595
:103390004E4B00AABB1234003412BBAA00254310C6
:1033A0001200E77EE300004222B6E900CC330008B9
:1033B00000000020A8000000602F000874340008FE
:1033C000A8000020585F0000702F000800000000D7
:1033D0000000000000000000D1D1E0D0000000009B
:1033E000D2D2000000000000000000000000000039
:1033F00000000000000000000000000000000000CD
:1034000000000000000000000000000000000000BC
:10341000000000000000313233343536373839319E
:1034200032333435363738390000000000000000F0
:10343000000000000000313233343536373839317E
:1034400032333435363738390000000000000000D0
:10345000000000000000000000000000000000006C
:103460000102030401020304060708090204060816
:043470000000000058
:0400000508000131BD
:00000001FF
